:100000000C9413050C943B050C943B050C943B0598
:100010000C943B050C943B050C943B050C943B0560
:100020000C943B050C943B050C94DB120C944A1386
:100030000C943B050C943B050C943B050C943B0540
:100040000C943B050C943B050C943B050C943B0530
:100050000C943B050C943B050C943B050C947C15CF
:100060000C943B050C943B050C943B050C943B0510
:100070000C943B050C943B050C943B050C943B0500
:100080000C94C6150C943B050C943B050C943B0555
:100090000C943B050C943B050C943B050C943B05E0
:1000A0000C943B050C943B050C943B0505A84CCDEA
:1000B000B2D44EB93836A9020C50B9918688083CA2
:1000C000A6AAAA2ABE000000803F2050545300591F
:1000D000455320284129002F0053484F54200050F9
:1000E0004C41594552200000000000003E5B4F5B30
:1000F0003E3E6B4F6B3E1C3E7C3E1C183C7E3C18CB
:100100001C577D571C1C5E7F5E1C00183C1800FFAE
:10011000E7C3E7FF0018241800FFE7DBE7FF3048DC
:100120003A060E2629792926407F050507407F05D6
:10013000253F5A3CE73C5A7F3E1C1C08081C1C3ECD
:100140007F14227F22145F5F005F5F06097F017FBB
:10015000006689956A606060606094A2FFA294085E
:10016000047E040810207E201008082A1C08081CA1
:100170002A08081E101010100C1E0C1E0C30383EE1
:100180003830060E3E0E06000000000000005F0042
:10019000000007000700147F147F14242A7F2A120E
:1001A00023130864623649562050000807030000F4
:1001B0001C2241000041221C002A1C7F1C2A080826
:1001C0003E08080080703000080808080800006039
:1001D000600020100804023E5149453E00427F4025
:1001E0000072494949462141494D331814127F1084
:1001F00027454545393C4A494931412111090736CE
:1002000049494936464949291E000014000000406A
:100210003400000008142241141414141400412264
:10022000140802015909063E415D594E7C12111213
:100230007C7F494949363E414141227F4141413E0F
:100240007F494949417F090909013E414151737F75
:100250000808087F00417F41002040413F017F089E
:100260001422417F404040407F021C027F7F0408EF
:10027000107F3E4141413E7F090909063E4151211F
:100280005E7F09192946264949493203017F010346
:100290003F4040403F1F2040201F3F4038403F63C9
:1002A0001408146303047804036159494D43007F23
:1002B0004141410204081020004141417F040201F4
:1002C0000204404040404000030708002054547896
:1002D000407F284444383844444428384444287FE4
:1002E000385454541800087E090218A4A49C787F3E
:1002F0000804047800447D40002040403D007F1009
:1003000028440000417F40007C047804787C080485
:1003100004783844444438FC182424181824241839
:10032000FC7C08040408485454542404043F442426
:100330003C4040207C1C2040201C3C4030403C4441
:10034000281028444C9090907C4464544C440008FD
:10035000364100000077000000413608000201022B
:1003600004023C2623263C1EA1A161123A404020F3
:100370007A3854545559215555794121545478416E
:10038000215554784020545579400C1E5272123930
:1003900055555559395454545939555454580000E9
:1003A000457C410002457D420001457C40F0292406
:1003B00029F0F0282528F07C545545002054547C21
:1003C000547C0A097F493249494932324848483207
:1003D000324A4848303A4141217A3A424020780036
:1003E0009DA0A07D39444444393D4040403D3C24DB
:1003F000FF2424487E4943662B2FFC2F2BFF09291D
:10040000F620C0887E090320545479410000447DC1
:10041000413048484A32384040227A007A0A0A720B
:100420007D0D19317D2629292F28262929292630B5
:10043000484D4020380808080808080808382F10D8
:10044000C8ACBA2F102834FA00007B000008142A28
:10045000142222142A14089500220095AA0055009F
:10046000AAAA55AA55AA000000FF00101010FF000C
:10047000141414FF001010FF00FF1010F010F014FF
:100480001414FC001414F700FF0000FF00FF141404
:10049000F404FC141417101F10101F101F14141450
:1004A0001F00101010F0000000001F101010101F8F
:1004B00010101010F010000000FF1010101010109D
:1004C000101010FF10000000FF140000FF00FF00DC
:1004D000001F10170000FC04F41414171017141454
:1004E000F404F40000FF00F714141414141414F7A7
:1004F00000F7141414171410101F101F141414F400
:10050000141010F010F000001F101F0000001F1446
:10051000000000FC140000F010F01010FF10FF1499
:100520001414FF141010101F00000000F010FFFF43
:10053000FFFFFFF0F0F0F0F0FFFFFF000000000011
:10054000FFFF0F0F0F0F0F38444438447C2A2A3E18
:10055000147E02020606027E027E02635549416352
:100560003844443C04407E201E2006027E0202994C
:10057000A5E7A5991C2A492A1C4C7201724C304AE5
:100580004D4D303048784830BC625A463D3E49496E
:1005900049007E0101017E2A2A2A2A2A44445F4416
:1005A0004440514A444040444A51400000FF010346
:1005B000E080FF000008086B6B0836123624360610
:1005C0000F090F060000181800000010100030403E
:1005D000FF0101001F01011E00191D1712003C3C04
:1005E0003C3C0000000000F0F89C8E8783878E9CC6
:1005F000F8F00000FEFF0303030303070EFCF800FE
:1006000000FEFF0303030303070EFCF80000FFFFD7
:1006100000000000000000FFFF0000FEFF83838356
:100620008383C7EE7C380000F8FC0E070303030742
:100630000EFCF800003F7FE0C08080C0E07F3FFFFD
:10064000FF01010101010101FFFF0000FFFF0C0C90
:100650000C0C1C3E77E3C100007FFFC0C0C0C0C0CF
:10066000E0703F1F00001F3F70E0C0C0C0E0703F5F
:100670001F00007FFFC1C1C1C1C1E3773E1C000064
:100680001F3F70E0C0C0C0E0703F1F0000000000CE
:1006900001FFFF01000000D5F08D14A1C881CFD962
:1006A000F1AF20004241434B20544F204D454E5561
:1006B00000524553544152542047414D4500524544
:1006C0005455524E20544F2047414D450008183C88
:1006D0003C3C180800183C7E7E7E3C18003C42A53D
:1006E00081A599423C2053544152545300504C41EF
:1006F000594552200028422920534B495000434F6E
:10070000494E20544F535300284229204241434B25
:1007100000284229204241434B004355524C494E48
:10072000472047414D45204D4144452042592054E2
:10073000554E43415920415948414E20207C2020AC
:100740004749544855423A2068747470733A2F2FC1
:100750006769746875622E636F6D2F54756E63617F
:1007600079417968616E2020200076312E302E3953
:10077000004355524C4455494E4F004F4646004F9A
:100780004E00544F47474C45202841290028422914
:10079000204241434B0041494D205346583A2000E6
:1007A0004F4646004F4E005346583A202020004FF7
:1007B0004646004F4E004D555349433A20002D2DDB
:1007C0002D2D2D2D2D2D2D2D2D2D2D2D2D00534548
:1007D0005454494E47530045524153454421004823
:1007E0004F4C442028412900284229204241434BB4
:1007F000002D2D2D2D2D2D2D2D2D2D2D2D2D2D2D56
:10080000004849474853434F52453A20002D2D2D6B
:100810002D2D2D2D2D2D2D2D2D2D2D2D00524553D2
:10082000554C5453003E414141227F4040407F7F20
:10083000091929467F404040407F4141221C7F40AA
:1008400040407F417F4100007F0618607F3E41416C
:10085000413E0505050505050305052842290083D8
:1008600000C800C400C800A500C800C400C80083B8
:1008700000C8000000C8008300C800A500C800C46C
:1008800000C800A500C800C400C8000000C800AF30
:1008900000C8008300C8006E00C8008300C8006E56
:1008A00000C8000000C800AF00C8008300C8006E88
:1008B00000C8008300C8006E00C8000000C80062C5
:1008C00000C8009300C800C400C8009300C800C45A
:1008D00000C8000000C8006E00C800A500C800DC09
:1008E00000C800A500C800DC00C8000000C800A5C2
:1008F00000C800C400C800AF00C8009300C800AF23
:1009000000C8009300C8008300C8006200C80093BC
:1009100000C8006200C8000000FA004241434B20BA
:10092000544F204D454E553F00524553544152546B
:100930002047414D453F00080B000202020000091C
:10094000040000010202000005240010010524013A
:100950000101042402060524060001070581031095
:10096000004009040100020A0000000705020240DD
:10097000000007058302400000040309041201007F
:1009800002EF0201404123368000010102030141D0
:10099000726475696E6F204C4C4300414250313394
:1009A0003036007E090909060000007F40404040C3
:1009B0000000007E0909097E00000003047804039A
:1009C0000000007F494949410000007F091929467C
:1009D00000000000427F400000000062514949468B
:1009E0000000003F4038403F000000417F410000D0
:1009F0000000007F0618607F000000464949493129
:100A000000000000005F00000000003E4141413E48
:100A10000000007F4040407F0000007F4141221CD9
:100A2000000000005A1611241FBECFEFDAE0DEBF2F
:100A3000CDBF11E0A0E0B1E0EEEAF6E502C005901E
:100A40000D92A238B107D9F726E0A2E8B1E001C0C3
:100A50001D92A73EB207E1F715E0C3E1D5E004C05F
:100A60002197FE010E94482BC231D107C9F70E948D
:100A700087160C94552B0C940000809182010895E8
:100A80004F925F926F927F928F929F92AF92BF929E
:100A9000CF92DF92EF92FF920F931F93CF93DF934A
:100AA000FB01E00FF11D1E161F060CF08AC060341A
:100AB00071050CF086C0DB0177FF04C0AA27BB27B5
:100AC000A61BB70BA770BB27EB0177FD2796E3E0CA
:100AD000D595C795EA95E1F777FF07C0219768E0BC
:100AE00070E0FB01EA1BFB0BDF0130E00695069589
:100AF0000695802E912C8A01AE015695542F4427DD
:100B000057954795480F591F4F575D4FBE01E0E875
:100B1000F0E07F01E81AF90A88E090E03C016A1AE7
:100B20007B0A6F3FFFEF7F070CF43BC090E080E053
:100B30005A01E0E8AE0EB11C6F3F760709F452C0CF
:100B4000FC01E00FF11FE4916A01C80ED91EF0E02C
:100B50002F010A2E01C0440C0A94EAF7F6015080D6
:100B6000452840821097B1F06730710599F0F8017F
:100B7000E80FF91FE4916501C80ED91EF0E02F01BE
:100B8000062C02C0559447940A94E2F7F60150806F
:100B9000452840820196821793071CF4E816F9064F
:100BA00059F66F5F7F4F020F131F40585F4FCB0105
:100BB0008C1B9D0B8815990524F46830710509F08C
:100BC000B0CFDF91CF911F910F91FF90EF90DF9009
:100BD000CF90BF90AF909F908F907F906F905F90DD
:100BE0004F900895109709F0C2CFD4CFE1E8F2E01A
:100BF000A0E0B8E000800EBC8111012C1197A0FD8F
:100C0000FDCF0192B9F70DB40895E1E0F0E00E9444
:100C10001A06319728F068517C4F8F4F9F4FF9CFBC
:100C2000AB01FC010E941A06641775078E079F0727
:100C3000C8F30895A7E6B2E02FB7F8947D918D919F
:100C40009C9166B52FBFA89B05C06F3F18F47F5FCE
:100C50008F4F9F4F22E0660F771F881F991F2A959D
:100C6000D1F70895FC0180918002882311F13FB7EC
:100C7000F89482E08093E9002091F200822F90E0C6
:100C80001816190614F481E090E0882339F02898AA
:100C900044E640937F024091F1004083222339F0E3
:100CA0002091F200211103C02BE62093E8003FBF02
:100CB00008958FEF9FEF08952FB7F89483E0809306
:100CC000E9009091E800892F807295FF04C090910F
:100CD000F20080E4891B2FBF089580917702811173
:100CE0000DC082E08093730284E0809374021092BE
:100CF00076021092750281E08093770283E792E09A
:100D000008958F929F92AF92BF92CF92DF92EF920F
:100D1000FF920F931F93CF93DF936C017B018A01A6
:100D200080911C01882309F458C080918002882397
:100D300009F453C08091720280FF05C08091E000E9
:100D400082608093E000E801B12C8AEFA82E93E046
:100D5000892E2AE3922E209711F4BB20B9F10E942C
:100D60005C06811106C0AA94AA20B9F10E9405066A
:100D7000F2CF8C171D0611F00CF08C2F9FB7F89452
:100D80008092E9002091E80025FD02C09FBFE3CFDB
:100D9000282F30E0C21BD30BF701815020F0419186
:100DA0004093F100FACFE20EF31EBB2021F09092A7
:100DB000E800B12CEBCF8091E80085FDE7CF909261
:100DC000E800BB24B394209709F3F3CF5D9884E641
:100DD00080937102101611063CF081E090E0F6015C
:100DE0009383828310E000E0C801DF91CF911F91CF
:100DF0000F91FF90EF90DF90CF90BF90AF909F90BA
:100E00008F900895CF93DF931F92CDB7DEB769839C
:100E1000DC01ED91FC910280F381E02D41E050E096
:100E2000BE016F5F7F4F09950F90DF91CF910895BD
:100E300083E08093E9008091F200882319F08AE32F
:100E40008093E80008950E945C0690E00895CF9397
:100E5000DF931F92CDB7DEB7FC018485958597FDA2
:100E600008C02FEF3FEF358724870F90DF91CF9198
:100E70000895CE0101960E943206019719F48981E6
:100E800090E0F3CF8FEF9FEFF0CF0F931F93CF93AF
:100E9000DF931F92CDB7DEB78C01FC018485958569
:100EA00097FF0BC0CE0101960E943206019771F4A4
:100EB000898190E0F80195878487F801848595857C
:100EC0000F90DF91CF911F910F9108958FEF9FEFBA
:100ED000F1CFFC018485958597FD0BC09FB7F894F1
:100EE00082E08093E9008091F2009FBF90E001963C
:100EF00008959FB7F89482E08093E9008091F20012
:100F00009FBF90E0089540916D0250916E02209134
:100F10006B0230916C0242175307B4F49091E800D1
:100F20009570E1F39091E80092FD19C08093F10073
:100F300080916D0290916E0201968F739927892B93
:100F400019F48EEF8093E80080916D0290916E020B
:100F5000019690936E0280936D0281E0089580E087
:100F60000895DF92EF92FF920F931F93CF93DF9339
:100F7000D82E8A01EB017B01E40EF51ECE15DF05AC
:100F800059F0D7FE12C0FE0184910E94830721967A
:100F90008111F4CF0FEF1FEFC801DF91CF911F91A7
:100FA0000F91FF90EF90DF9008958881EECF0F931F
:100FB0001F93CF93DF931F92CDB7DEB782E0898373
:100FC00042E450E067E379E080E80E94B1070E94C4
:100FD0006D06DC0112960D911C910115110589F029
:100FE000D801ED91FC910280F381E02DBE016F5F8D
:100FF0007F4FC801099597FD04C0F8010085118550
:10100000ECCF89810F90DF91CF911F910F910895BF
:10101000615030F02091F100FC0120830196F8CF5F
:10102000289884E680937F020895AF92BF92CF9272
:10103000DF92EF92FF920F931F93CF93DF936C0198
:101040007B018B01040F151FEB015E01AE18BF0879
:10105000C017D10759F06991D601ED91FC9101902B
:10106000F081E02DC6010995892B79F7C501DF9143
:10107000CF911F910F91FF90EF90DF90CF90BF9095
:10108000AF90089520918A01E0918801F091890143
:10109000CF0102969093890180938801222319F051
:1010A000859194910895808191810895E1E7F0E020
:1010B00080818D7F8083109291004698479810928E
:1010C00087010895CF92DF92EF92FF92CF93DF9343
:1010D0000E944208811520E8920741F4DF91CF91E8
:1010E000FF90EF90DF90CF900C94560821E0209372
:1010F0008701813020E8920751F480918501909119
:10110000860190938901809388010E94420897FD8F
:1011100005C020918401222309F45BC02091830142
:10112000211157C021E020938B01EC01DF7720973C
:1011300009F052C081E080938C0146983FE9C32EAC
:101140003FE0D32EE12CF12CCAEFD0E0E091E10694
:10115000F091E2060995811103C081E080938C0132
:1011600080918B01882329F080918C01882309F4D8
:1011700046C047980E944208009709F444C09C0169
:10118000DE010E94F627DC01CB0129E0B595A79589
:10119000979587952A95D1F7109290002AE0209391
:1011A0009100D0929900C092980080938D01909305
:1011B0008E01A0938F01B0939001809171008260A5
:1011C00080937100DF91CF91FF90EF90DF90CF90EF
:1011D000089510928B01A9CF9E0150E040E060E499
:1011E00072E48FE090E00E94A22769017A0181E019
:1011F000C81AD108E108F10810928C01A7CF4699CE
:10120000B8CF479AB7CF8FEF9FEFDC01C5CF9C01D6
:10121000E1E7F0E090819D7F908310928A01E3EDF9
:10122000F6E0F0938901E0938801F0938601E09362
:101230008501318320837383628380E090E8958306
:1012400084830C9462082D9A0895BC0190E080E09C
:10125000AB01FC010E941A0641505109E109F10954
:1012600028F068517C4F8F4F9F4FF6CFAB01FC01A8
:101270000E941A06641775078E079F07C8F3089522
:101280008FB18095807F669B88601C9B84600895E9
:10129000109282013E983F9808953E9A3F9A81E0CD
:1012A000809382010895480F592F511D1416150679
:1012B000D4F580389105BCF597FF02C090E080E03E
:1012C0004138510514F040E850E0481BFB0177FD20
:1012D000379633E0F595E7953A95E1F7F695FE2FC9
:1012E000EE27F795E795E80FF91FEF57FD4F677069
:1012F000772781E090E001C0880F6A95EAF7382FE0
:10130000213041F4415078F08191DF011197832B16
:101310008C93F8CF8095415030F09191DF01119777
:1013200098239C93F8CF08952F923F924F925F920B
:101330006F927F928F929F92AF92BF92CF92DF92E5
:10134000EF92FF920F931F93CF93DF93CDB7DEB74A
:101350002E970FB6F894DEBF0FBECDBF6B015A01BA
:101360003E872D87261737070CF007C1E616F706CC
:101370000CF41BC1621773075CF03C2D2D2DCD843E
:10138000DE843D872E87382F292FC501A32EB22E4C
:10139000CE14DF04A9F5A816B90654F0382F292F6A
:1013A0008A159B0514F43A2D2B2D5C01832F922F67
:1013B0000A151B052CF0801791070CF4C801850154
:1013C0008F5F482F401B21E0B601C8012E960FB653
:1013D000F894DEBF0FBECDBFDF91CF911F910F916B
:1013E000FF90EF90DF90CF90BF90AF909F908F9045
:1013F0007F906F905F904F903F902F900C94530987
:10140000302F212F8C01832F922F3E2D2F2D7601EF
:10141000C32ED22E9501201B310B38872F834D858B
:101420005E854E195F095A8749873C01601A710A27
:1014300096012E193F093A832983AC014A195B09A9
:101440005C834B83C6012D853E85821B930B9C8755
:101450008B87C216D30609F443C0215031093E835D
:101460002D834701512C412C312C212C4D815E8143
:1014700048155905C4F1C10169857A850E94342B4C
:10148000FB01E00FF11FC20169817A810E94342BB8
:10149000600F711F8F819885280E391E460C571CCE
:1014A0006E177F071CF49E2FFB01692F90E48916AD
:1014B000910444F46F5F462F4E1B21E0B401CF012D
:1014C0000E9453092FEF821A920AD0CF3A2D2B2D6A
:1014D0005C01832F922F3C2D2D2DCD84DE8474C092
:1014E000DE82CD82BECFC4014D855E85841B950B07
:1014F0004B815C81849F9001859F300D949F300DBE
:1015000011243E832D83C4018E199F09869D70018D
:10151000879DF00C969DF00C1124C814D9040CF48E
:1015200056C08D819E816B857C850E94342BFB018A
:10153000EA0DFB1DC70169817A810E94342B600F7F
:10154000711F8D819E812B813C81820F931F9E8311
:101550008D83E60CF71C6E177F071CF49E2FFB0192
:10156000692F6F5F462F4E1B21E0B401CF010E940F
:1015700053093FEF831A930AD0CF4D855E85E41659
:10158000F5060CF005CFE616F7060CF49FCF302FCA
:10159000212F85015C01832F922F3D852E857E872B
:1015A0006D876701E32EF22EE8CE2D853E85E2168B
:1015B000F3060CF42FCF302F212F8501A32EB22E4E
:1015C0003E2D2F2DED84FE843D872E8723CF2E9632
:1015D0000FB6F894DEBF0FBECDBFDF91CF911F9144
:1015E0000F91FF90EF90DF90CF90BF90AF909F90C2
:1015F0008F907F906F905F904F903F902F900895C5
:1016000090915802982329F490915902982381E0EF
:1016100009F480E00895CF93C82F0E944009982FC5
:101620009C2381E09C1380E0CF91089580E00C948E
:10163000F60580389105B8F460347105A0F420E116
:1016400091E061FD94E060FD990F62FD9295687FE5
:10165000269FD0011124A80FAF57BD4F8C9140FF9A
:1016600003C0892B8C93089590958923FBCF2F92EB
:101670003F924F925F926F927F928F929F92AF9222
:10168000BF92CF92DF92EF92FF920F931F93CF936F
:10169000DF9300D000D0CDB7DEB77C018B01242FC3
:1016A00030E03C832B8381E090E05C01A21AB30A16
:1016B0001901319421943108220C331CB901600FB7
:1016C000711F41E0C7010E94190BB8018B819C81F9
:1016D000681B790B41E0C7010E94190B41E0B8017A
:1016E0008B819C818E0D9F1D0E94190B41E0B801DA
:1016F000C7012B813C81821B930B0E94190B81E057
:1017000090E09A838983D12CC12CB7FC0BC02B812C
:101710003C81215031093C832B8332E0230E311C64
:10172000A20CB31C8FEFC81AD80A29813A812E5F08
:101730003F4F3A832983A20EB31E36016E0C7F1CE5
:1017400041E08B809C80800E911EB401C3010E94F9
:10175000190B27014C185D0841E0B401C2010E9439
:10176000190B41E048018B819C81881A990AB401C8
:10177000C3010E94190B41E0B401C2010E94190B80
:101780004601800E911E41E0B4016B807C806E0C9E
:101790007F1CC3010E94190B41E0B40127012B817A
:1017A0003C81421A530AC2010E94190B48018C184D
:1017B0009D0841E0B401C3010E94190B41E0B4014E
:1017C000C2010E94190B8B819C81C816D9060CF4AA
:1017D0009CCF0F900F900F900F90DF91CF911F91A2
:1017E0000F91FF90EF90DF90CF90BF90AF909F90C0
:1017F0008F907F906F905F904F903F902F900895C3
:101800006F927F928F929F92AF92BF92CF92DF9210
:10181000EF92FF920F931F93CF93DF936D3089F078
:10182000C0905602D09057026A30E1F410925502EF
:101830001092540288E0C80ED11CD0925702C09278
:10184000560281E090E0DF91CF911F910F91FF90C0
:10185000EF90DF90CF90BF90AF909F908F907F9050
:101860006F90089560900101E0905402F09055024D
:10187000E5E06E9FE0011124C951DF4F570100E000
:1018800010E0053029F0CE010196FE011491EC0123
:10189000460188E0782E412F417010FD1BC0662064
:1018A00021F0B401C5010E94190B16957A94FFEF3F
:1018B0008F1A9F0A7110EFCF0F5F8FEFA81AB80A27
:1018C0000630F1F6E6E0EE0EF11CF0925502E092E1
:1018D0005402B7CF462DE5CF0F931F93CF93DF93DD
:1018E0008C01D0E0C0E0F801EC0FFD1F649166238D
:1018F00041F083EE96E00E94000C892B11F02196B6
:10190000F2CFCE01DF91CF911F910F910895DF9219
:10191000EF92FF920F931F93CF93DF937C01D22E10
:101920008B01040F111DEB0177FF02C0D0E0C0E076
:10193000C8010134110514F080E490E0C817D907FC
:101940003CF44D2DBE01C7010E94190B2196F0CF2A
:10195000DF91CF911F910F91FF90EF90DF9008954D
:101960007F928F929F92AF92BF92CF92DF92EF922F
:10197000FF920F931F93CF93DF93EC018B01742E93
:101980007B0182E0E81AF108242F45E0B701CE017F
:101990000E94870C5E018FEFA81AB80A272D45E038
:1019A000B701C5010E94870C015011094E0182E068
:1019B000880E911C272D43E0B801C4010E94870CBA
:1019C0006E0181E0C81AD108272D45E0B701C60194
:1019D0000E94870C2297272D43E0B801CE010E9478
:1019E000870C272D43E0B801C4010E94870C272DE6
:1019F00045E0B701C5010E94870C272D43E0B801DF
:101A0000CE010E94870C272D45E0B701C601DF916A
:101A1000CF911F910F91FF90EF90DF90CF90BF90EB
:101A2000AF909F908F907F900C94870CCF92DF9215
:101A3000EF92FF920F931F93CF93DF936B01122FBF
:101A4000EC017C01E40EF11CCE15DF0544F4202FDF
:101A5000412FB601CE010E94870C2196F5CFDF9170
:101A6000CF911F910F91FF90EF90DF90CF9008954D
:101A7000CF92DF92EF92FF920F93CF93DF936C019F
:101A80007B01C42FD22F6034710520F4202FC601B2
:101A90000E945309B7016D0F711D615071096034C7
:101AA000710528F4202F4C2FC6010E945309202FC6
:101AB0004D2FB701C6010E94870CC6018C0F911DE6
:101AC000202F4D2FB7010197DF91CF910F91FF90FC
:101AD000EF90DF90CF900C94870C0F931F93CF93D0
:101AE000DF9380915C0290915D02059751F48091A3
:101AF0003C0290913D02A091A601B091A7010197EF
:101B000021F0A091A401B091A5012EE330E00E9444
:101B10004E2B24E630E040E050E00E94A227122F36
:101B2000C22FD32F01E026E04CE769E370E082E0AA
:101B300090E00E94380D1C161D0694F424E0412FFD
:101B40006AE370E080E490E08C1B9D0B0E94160D10
:101B500024E0412F6AE370E080E490E00E94160DDB
:101B600021E046E069E370E080E490E0DF91CF910E
:101B70001F910F910C94870C0F931F93CF93DF93BA
:101B800000915E02002E000C110B0E5D1F4FC091E4
:101B90005F020C2E000CDD0BC459DF4F4EE0B80184
:101BA000CE010E94370B49E0B801CE010E94370BED
:101BB00044E0B801CE01DF91CF911F910F910C94B9
:101BC000370B0F9360915E02062E000C770B625F5D
:101BD0007F4F80915F02082E000C990B01E028E2F4
:101BE0004CE702960E94380D0F910895E0913F0254
:101BF00082E1E89FF0011124E855FE4F80E090E07B
:101C0000A0E8B1E480839183A283B383809105012E
:101C100090910601A0910701B091080184839583FA
:101C2000A683B783108611861286138614861586BE
:101C3000168617868091A301808B81E0818B10929C
:101C400038021092390210923A0210923B0210921E
:101C50003D0210923C02089522E030E0309355029C
:101C60002093540226E330E030935702209356022B
:101C70000C946C0CCF93DF93C0913F0282E1C89F1C
:101C8000E0011124C855DE4F688579858A859B85DA
:101C90009F772DEC3CEC4CE45DE30E94D1291816B3
:101CA0009CF06C857D858E859F859F77C1E02DECAE
:101CB0003CEC4CE45DE30E94D12918160CF0C0E026
:101CC0008C2FDF91CF910895C1E0FACF089590E075
:101CD00080E008958F929F92AF92BF920F931F93CF
:101CE000CF93DF93CDB7DEB7A1970FB6F894DEBFE1
:101CF0000FBECDBF19A2423008F44AE08E010F5D3D
:101D00001F4F842E912CB12CA12CA50194010E946F
:101D1000D427E62FB901CA01EA3044F5E05DD801C5
:101D2000EE938D01232B242B252B79F790E080E077
:101D3000109769F0FD0101900020E9F73197AF019C
:101D40004A1B5B0BBD0183EE96E00E941508A1962D
:101D50000FB6F894DEBF0FBECDBFDF91CF911F91BC
:101D60000F91BF90AF909F908F900895E95CD7CF6F
:101D7000CF92DF92EF92FF92CF93DF936B017C01C2
:101D80006DE283EE96E00E94000CEC016627772757
:101D9000CB016C197D098E099F094AE00E946A0EE9
:101DA0008C0F9D1FDF91CF91FF90EF90DF90CF9030
:101DB0000895009769F0FC0101900020E9F7319740
:101DC000AF01481B590BBC0183EE96E00C9415083B
:101DD00090E080E0089543E0843691052CF441E0E2
:101DE0008A3091050CF042E028E630E056E0459F4D
:101DF000201931091124309355022093540226E30F
:101E000030E03093570220935602BC01990F880BA3
:101E1000990B97FF06C00E94B80E8AEC90E00C94D4
:101E20006C0C4AE00E946A0EF8CFBC01990F880B37
:101E3000990B97FD0C94B80E4AE00C946A0EEF9241
:101E4000FF920F931F93CF93DF93E091A301D1E013
:101E5000DE0FF0E0EF55FE4F6081C1E0C60F8091CC
:101E60008106909182066CE370E00E94202B7B013A
:101E700081E0E822FF2400E02EE040E870E060E02E
:101E800090E080E00E94160DEF2809F448C001E0C0
:101E90002EE04EE370E060E082E090E00E94160DDC
:101EA0001092010188E090E09093550280935402D3
:101EB00003E010E010935702009356028FED90E07C
:101EC0000E946C0C6D2F70E090E080E04AE00E9470
:101ED0006A0E81E08093010186E490E090935502C0
:101EE00080935402109357020093560289ED90E0BC
:101EF0000E946C0C6C2F70E090E080E04AE00E9441
:101F00006A0E87ED90E00E946C0C84E090E0DF9117
:101F1000CF911F910F91FF90EF900C94150F81E0DE
:101F200080930101BFCF6F927F928F929F92AF9269
:101F3000BF92CF92DF92EF92FF920F93CF93DF93F6
:101F4000E82ED62EF72E3A01C22F609181067091AD
:101F5000820690E080E00E941F292AE037ED43EAE4
:101F60005DE30E94D6294B015C016C2F70E090E08C
:101F700080E00E9421292AE939E949E15FE30E94D2
:101F8000D6299B01AC01C501B4010E9406280E941C
:101F9000432A9B01AC010E9406280E94E928660E94
:101FA000771E28E0E29EC0011124CD2DDF2D912C5B
:101FB000812C9C012D55364F7901F701E80DF91D53
:101FC000E491D12CC12CAE2EB12CC5010C2C02C039
:101FD000959587950A94E2F780FF0BC0B601660FCE
:101FE000771F660D771D01E022E042E0CE010E94DE
:101FF000160D3FEFC31AD30A87E0C816D10429F79C
:102000002FEF821A920A229635E083169104A9F6E0
:10201000DF91CF910F91FF90EF90DF90CF90BF9025
:10202000AF909F908F907F906F9008950C948C2725
:102030001F93CF93DF93EC01162F0E948C27181764
:1020400039F0612FCE01DF91CF911F910C9494272D
:10205000DF91CF911F9108958F929F92AF92BF927F
:10206000CF92DF92EF92FF926B017C01C216D306F2
:10207000E406F50684F449015A018C189D08AE085F
:10208000BF080E942B27A50194010E94A227C60E1B
:10209000D71EE81EF91EC701B601FF90EF90DF9032
:1020A000CF90BF90AF909F908F9008952F923F92C6
:1020B0004F925F926F927F928F929F92AF92BF9258
:1020C000CF92DF92EF92FF920F931F93CF93DF9304
:1020D000CDB7DEB760970FB6F894DEBF0FBECDBFA9
:1020E000188A80913F022889821708F44EC1022F76
:1020F00010E032E1309FC001319F900D1124AC01FE
:1021000048555E4F7A01DA0151968C915197882398
:1021100009F437C16D917D918D919C910E94E928C0
:1021200020915F02022E000C330BF901E60FF71F1E
:10213000FC83EB83D70114966D917D918D919C91D9
:1021400017970E94E92820915E02022E000C330BA3
:10215000F901E60FF71FFA83E983D70150968C91B6
:102160008111F8C041E0BF018B819C810E94B00CBD
:102170008090A4019090A501B2E08B1691040CF41C
:1021800000C122E1209FF001219FF00D1124E855AC
:10219000FE4F60857185828593859F77248535857F
:1021A000468557855F770E9406286B017C012AE9E6
:1021B00039E949E95EE30E94D12918160CF0E1C023
:1021C000092C000CAA08BB0831E0831A9108A10869
:1021D000B108C501B40152E0660F771F881F991F2F
:1021E0005A95D1F723E630E040E050E00E94A22764
:1021F0002F5F2987A701960160E070E080E090E4FE
:102200000E9405286B017C012AE939E949E15FE375
:102210000E94722887FDA6C020E030E040E050E434
:10222000C701B6010E94D12918160CF4A4C0C5013B
:10223000B401660F771F881F991F23E630E040E046
:1022400050E00E94A227312C212C42E1409FC00186
:10225000419F900D112488559E4FDC011896BD8733
:10226000AC87FC013C96FF87EE8730E04901FFEF29
:102270008F1A9F0A092C000CAA08BB0831952195DA
:102280003109C901330FAA0BBB0B8D839E83AF832A
:10229000B8879985291608F074C0AFEF2A1A3A0A50
:1022A000229CB001239C700D700D1124072E000C90
:1022B000880B990B0E9421292DEC3CEC4CEC5EE341
:1022C0000E94D6292B013C01EC85FD8520813181BE
:1022D00042815381C701B6010E94D629A301920110
:1022E0000E94D6290E94E9282B813C81261B370BAE
:1022F0003B872A87AE85BF852D913D914D915C919D
:10230000C701B6010E94D629A30192010E94D629D5
:102310000E94E92809811A81061B170BA501940167
:102320006D817E818F8198850E942C102B01A501E3
:1023300094016D817E818F8198850E942C10400EC2
:10234000511E8A859B85860F971F41E0B2010E942E
:10235000190B9FCF42E069817A818B819C810E9419
:10236000370B06CF4AE9C42E49E9D42E49E1E42EC1
:102370004FE3F42E5CCFC12CD12CE12C30E4F32EB2
:1023800056CFB889BF5FB88BACCE60960FB6F894C5
:10239000DEBF0FBECDBFDF91CF911F910F91FF9098
:1023A000EF90DF90CF90BF90AF909F908F907F90F5
:1023B0006F905F904F903F902F9008950E94560825
:1023C000109253021092520282EE9FEF90930F01EF
:1023D00080930E0110924F0210924E021092500202
:1023E000809148029091490222E0009709F421E08F
:1023F000209302011092A2011092A1011092A0015B
:1024000010929F0110929E0110929D0110923F0226
:102410001092A3011092B9011092CB011092DD012C
:102420001092EF01109201021092130210922502F5
:1024300010923702019761F50E941A066115710525
:102440008105910511F00E947A270E942B2722E036
:1024500030E040E050E00E94A22721E0672B682B8B
:10246000692B09F420E020939B01109297011092B0
:102470009A01109299011092960110929501109272
:10248000980184E090E090935D0280935C0208954F
:102490000E94F60D85E090E0F6CFEF92FF920F9349
:1024A0001F93CF93DF9300D000D000D01F92CDB701
:1024B000DEB77C0101E020E440E870E060E090E0FD
:1024C00080E00E94160D1092010100E02CE140E630
:1024D00062E170E080E190E00E94380DC7010E9447
:1024E000832720E830E0A90166E0869F4019510962
:1024F0001124CA0157FD0196959587959093550231
:102500008093540208E110E01093570200935602A2
:10251000C7010E946C0C87E0E0E5F1E0DE01119656
:1025200001900D928A95E1F71093550200935402A1
:1025300002E210E01093570200935602CE0101967A
:102540000E94D90E84E490E0909355028093540247
:1025500010935702009356028FEC90E00E946C0C8F
:1025600081E08093010127960FB6F894DEBF0FBE7D
:10257000CDBFDF91CF911F910F91FF90EF90089504
:10258000CF93DF93EC010E9483272AE730E096E0A7
:10259000899F201931091124309355022093540248
:1025A00086E390E09093570280935602CE01DF912C
:1025B000CF910C946C0C1F920F920FB60F921124B6
:1025C0008F939F938091E1009091E100937F90938E
:1025D000E10083FF0FC01092E90091E09093EB00BF
:1025E0001092EC0092E39093ED001092800298E03C
:1025F0009093F00082FF22C093E09093E9009091C5
:10260000F200992319F09AE39093E80090917102F7
:10261000992341F090917102915090937102911120
:1026200001C05D9A90917F02992341F090917F02C1
:10263000915090937F02911101C0289A84FF18C095
:102640008091E2008E7E81608093E2008091E100C3
:102650008F7E8093E100809172028E7E80618093F4
:1026600072029F918F910F900FBE0F901F9018953F
:1026700080FFF7CF8091E2008E7E80618093E20040
:102680008091E1008E7E8093E100809172028E7EC7
:102690008160E5CF1F920F920FB60F921124CF9257
:1026A000DF92EF92FF920F931F932F933F934F93DD
:1026B0005F936F937F938F939F93AF93BF93EF93AA
:1026C000FF93CF93DF93CDB7DEB76C97DEBFCDBF5F
:1026D0001092E9008091E80083FF25C068E0CE01F8
:1026E00045960E94080882EF8093E8008D8987FF55
:1026F00039C09091E80090FFFCCF982F907609F0B8
:1027000034C19E894F89588D2F89F88C911131C021
:10271000803861F5809170028093F1001092F10091
:102720008EEF8093E8006C960FB6F894DEBF0FBE74
:10273000CDBFDF91CF91FF91EF91BF91AF919F916D
:102740008F917F916F915F914F913F912F911F9149
:102750000F91FF90EF90DF90CF900F900FBE0F90F2
:102760001F9018959EEF9093E800C7CF1092F1004C
:10277000D5CF913059F48111D3CF4130510581F635
:10278000809170028D7F80937002CACF933049F49C
:102790008111C6CF4130510519F6809170028260D7
:1027A000F2CF953041F48091E80080FFFCCF2068A3
:1027B0002093E300B5CF963009F0A9C00B8D1C8D96
:1027C00022E01092E90010926E0210926D02F21255
:1027D0002EC010926C0210926B020E94D7071F82CB
:1027E00099E09983FA8291E09E8390EA98879AEF24
:1027F000998720916D0230916E02275F3F4F3C8395
:102800002B838D831092E90010926E0210926D025C
:1028100010936C0200936B0249E050E0BE016F5FC1
:102820007F4F80E00E94B1070E94D70779CF1093B5
:102830006C0200936B020E946D06DC0112960D91F2
:102840001C910115110509F451C1D801ED91FC91BC
:102850000480F581E02DBE016B5E7F4FC8010995B4
:10286000009709F03EC1F80100851185EACFF3E039
:10287000FF120EC08F89882309F440C0823061F4B2
:1028800040E867E08BE999E00E942716811148CF64
:1028900081E28093EB0047CF813029F440E86BE080
:1028A0008FE899E0F1CF833099F70E946D06DC0143
:1028B0001296ED90FC908E010F5F1F4F6801E1149E
:1028C000F10479F0D701ED91FC910680F781E02DBC
:1028D000B801C7010995080F111DF701E084F184C3
:1028E000EECFD8011C92F60101900020E9F7319754
:1028F000BF016C197D0940E0C601C6CF69E779E0E8
:10290000FB01449150E080E80E94B10709CF973065
:1029100009F4BECF983021F481E08093F10000CF1C
:10292000993009F0FDCE837009F0B2CFECE2F1E00E
:1029300081E031E096E32191222371F08093E90058
:102940003093EB00DF0111972C912093EC009093D2
:10295000ED008F5F873079F78EE78093EA00109261
:10296000EA008F8980938002DBCE8B8D9C8D109244
:10297000E90010926E0210926D0290936C028093A7
:102980006B02898D811192C08E899D89913A49F49B
:10299000813209F07DCF47E050E065E171E080E0F1
:1029A000B3CF913209F074CF833269F48F89988D57
:1029B000B0E0A0E08093110190931201A093130165
:1029C000B0931401ADCE803269F48091E80082FFAB
:1029D000FCCF67E085E191E00E9408088BEF8093CF
:1029E000E8009ECE823209F09BCE8F8980931C0135
:1029F000EEEFFFE7859194918B3F9C4D51F1E0E024
:102A0000F8E08091150190911601A0911701B09105
:102A10001801803B9440A105B105F1F480911C019F
:102A200080FD1AC0EE3F8AE0F80789F587E797E74F
:102A3000918380838091600080936F0288E19BE0A6
:102A40000FB6F894A895809360000FBE9093600035
:102A500067CEEEEFFAE0D5CF808191818737974737
:102A600009F05ECEA8958091600088618093600037
:102A700080916F0280936000EE3F2AE0F20789F0B8
:102A80008091FE0A9091FF0A9183808349CE8081D4
:102A900091818737980751F29093FF0A8093FE0A3D
:102AA000C5CF1092FF0A1092FE0A3ACE0E946D0620
:102AB000DC0112960D911C910115110509F4E8CE67
:102AC000D801ED91FC910190F081E02DBE016B5E8B
:102AD0007F4FC8010995811123CEF801008511852A
:102AE000EBCF181619060CF41BCED2CEF1E0FF1274
:102AF000BECE6DE779E004CF0F920FB68F939F9310
:102B0000EF93FF93809162028D5F8D3708F08D57B0
:102B100080936202E3E6F2E080818E4F80839181B0
:102B20009F4F918382818F4F828383818F4F8383D5
:102B3000E7E6F2E080818F5F808381818F4F818320
:102B400082818F4F828383818F4F83838FB18F6088
:102B500066991C9B88278F3681F480916102981BAF
:102B6000963068F0E0E0F8E087E78083818388E1D1
:102B700080936000F0936000FFCF90936102FF911B
:102B8000EF919F918F910FBE0F9018951F920F920A
:102B90000FB60F9211242F933F934F935F936F9330
:102BA0007F938F939F93AF93BF93EF93FF93809106
:102BB0008D0190918E01A0918F01B0919001892B90
:102BC0008A2B8B2B09F440C080918C0181110BC0A2
:102BD00088B190E4892788B980918B01882319F006
:102BE00088B1805888B980918D0190918E01A09113
:102BF0008F01B0919001181619061A061B069CF455
:102C000080918D0190918E01A0918F01B0919001E2
:102C10000197A109B10980938D0190938E01A09332
:102C20008F01B0939001FF91EF91BF91AF919F9170
:102C30008F917F916F915F914F913F912F910F9065
:102C40000FBE0F901F9018950E946208ECCFEF9274
:102C5000FF920F931F93CF93DF93F82E192FE62E39
:102C6000042F81E0860F880F0E94830783E00E9473
:102C70008307CF2DD12FEC0EFD2EF11CCE15DF05D5
:102C8000B9F007FF13C0FE0184910E948307182F3B
:102C900080E00E948307812321968111EFCFDF918D
:102CA000CF911F910F91FF90EF9008958881EDCF04
:102CB00081E0F5CFE3E8F6E01382128288EE93E03C
:102CC000A0E0B0E084839583A683B78386E391E098
:102CD000918380838FEF9FEF95878487E3EEF6E003
:102CE0001382128288E491E0918380838DE395E0E2
:102CF0009093E2068093E10680E090E89093E006EE
:102D00008093DF0646983E9A47983F9A0895CDB73C
:102D1000DEB7A897DEBFCDBF789483E084BD83E0A3
:102D200085BD81E080936E00E1E8F0E083E0808380
:102D3000E0E881E08083E1E983E08083E0E981E00D
:102D40008083E1EC87E08083E3EC81E08083E0EC4A
:102D500082E08083E2EC81E08083EAE787E08083A1
:102D6000806880831092800210927002109272022A
:102D70008091D70081608093D70080EA8093D8004B
:102D800089B5806189BD89B5826089BD09B400FEBD
:102D9000FDCF0E9405068091D8008F7C80618093D2
:102DA000D8008091E000807F8093E0008091E10076
:102DB0008E7E8093E1008DE08093E200559A209A08
:102DC00081EC80937C0085B1806F85B984B1877E6A
:102DD00084B984B1876E84B95E9A5F988AB1806D38
:102DE0008AB9769A6E9881B3806F81BB899880B3D7
:102DF0008D7080BB80E58CBD81E08DBD85E090E06D
:102E00000E9425095F9A85E090E00E9425095E985E
:102E10005C98E7E9F6E084EA96E024912EBD000094
:102E20000DB407FEFDCF31968E179F07B1F75C9A60
:102E300081E88093640080916500816080936500E3
:102E40000E94160B80E80E940B0B882381F05C988F
:102E500085EA8EBD00000DB407FEFDCF5C9A2E986A
:102E60002F982D9881E083BF889513BEFCCF84E016
:102E70000E940B0B882309F448C02D9884E80E9417
:102E80000B0B8823E1F00E94230988EC90E00E945C
:102E900025092F9882E090E00E948C278F3F29F02F
:102EA0006FEF82E090E00E94942784EF91E00E940F
:102EB00025092F9A84E80E940B0B8111FBCF84E136
:102EC0000E940B0B8823E1F00E94230988EC90E01C
:102ED0000E9425092E9882E090E00E948C2788238A
:102EE00029F060E082E090E00E94942784EF91E076
:102EF0000E9425092E9A84E10E940B0B8111FBCFC1
:102F000088EC90E00E942509B2CF0E94230982E05C
:102F100090E00E941610882309F46EC00E944D09AB
:102F200081E090E00E941610182F147081FF10C0ED
:102F300011112E9871EFE72EFF24FA9480E40E947D
:102F40000B0B882309F45BC02E9A2F9A0E94230949
:102F500082E390E00E9425090E9440098111F8CF88
:102F600080E18093000190E080E00E94161090E0E4
:102F7000909346028093450281E090E00E941610F3
:102F8000082F81E0011101C080E08093100182E0F0
:102F900090E00E941610182F81E0111101C080E00E
:102FA00080930D0183E090E00E94161091E0811162
:102FB00001C090E090930B01011103C0112309F4AB
:102FC0007BC00E944D098FB7F894409163025091E5
:102FD000640260916502709166028FBF1091930147
:102FE000112309F46CC01092930180E090E0892BCA
:102FF00051F30E940000E7CF0E94480991CF1123AE
:1030000031F024E0E216F10411F42E9A2F9881E0B9
:103010000E94F60500E128E547EE55E0B70184E19E
:1030200090E00E9440050E94160B8FE090E00E9405
:1030300025093FEFE31AF30A89E1E816F10409F0E4
:103040007DCF112311F02F9A2D9880E991E00E94F5
:1030500025090E94230981E090E00E94161080FF5C
:1030600077CF8AE090E00E9416109FEF980F9E3F66
:1030700008F06ECF22E330E03093550220935402E3
:1030800028E330E030935702209356020BE010E023
:10309000682F83EE96E00E94000CC8010E94161073
:1030A0000F5F1F4F0131110599F70E94160B88EE33
:1030B00093E00E9425094CCF0E94480984CF80915B
:1030C0009401942F981B892F90910001891748F43F
:1030D0008F5F891708F089CF81E083BF889513BE81
:1030E00084CF81E08093930140939401809191017A
:1030F0009091920101969093920180939101809119
:103100005902809358020E94400980935902E1E8D5
:10311000F2E011111FEF00241193119311931193F9
:103120000394D1F710925702109256021092550252
:103130001092540260916002662309F460C06150ED
:103140006093600270E09B012F5F3F4F032E000CE5
:10315000440B550B719561957109072E000C880B76
:10316000990B0E942C1060935F026091600270E0E6
:103170009B012F5F3F4F032E000C440B550B7195A5
:1031800061957109072E000C880B990B0E942C1079
:1031900060935E02809181069091820601969093E1
:1031A00082068093810680915C0290915D02049773
:1031B00078F480911001882359F080915202909107
:1031C0005302009709F101979093530280935202A2
:1031D000E0915C02F0915D02EB30F10508F0E1C195
:1031E000EC50F74E0C94482B2F19231B041C101D78
:1031F000C724891DF11EFA23BF2550266F26109281
:103200005F0210925E02C6CF20915102E22FF0E0E1
:10321000EE0FFF1FE15AF74F8591949132E0320F84
:10322000309351022F5FE22FF0E0EE0FFF1FE15AC3
:10323000F74F05911491B8010E94070964E01695B3
:1032400007956A95E1F7109353020093520280911B
:1032500051028E3508F4BCCF10925102B9CF809143
:103260005002811115C020910E0130910F01809103
:103270004E0290914F02019690934F0280934E021E
:10328000280F391F37FF90C130930F0120930E0193
:103290001091470282E090E07C01E11AF1081E14CF
:1032A0001F041CF0EE24E394F12C4BE558E0E2E51A
:1032B000F8E030E020E0849190E001968E9DB0012E
:1032C0008F9D700D9E9D700D1124260F371F319616
:1032D0004E175F0781F780E890E0821B930B97FD04
:1032E00001961C013594279480910E0190910F0155
:1032F000DC011296BA8BA98BE2E5F8E0FC87EB873C
:10330000512C412CED8660918106709182062B85AF
:103310003C8522553840690180915002882309F488
:103320006CC190E080E00E941F292AE037ED43EA5B
:103330005DE30E94D6294B015C01B601DD0C880BD0
:10334000990B0E9421292AE939E949E15FE30E94AA
:10335000D6299B01AC01C501B4010E9406280E9438
:10336000432A9B01AC010E9406280E94E928898912
:103370009A89860F971F988F8F8B4101D12CC12C72
:10338000D201AB5DB74FBC8BAB8BEB89FC89EC0DED
:10339000FD1DE4916F88788CB12CA12C2E2F30E08C
:1033A0003A8F298F898D9A8D0A2C02C09595879521
:1033B0000A94E2F780FF07C001E02D85422FB30198
:1033C000C4010E94160D3FEFA31AB30A6E0C7F1CB6
:1033D00087E0A816B10431F79FEFC91AD90A8E0CFD
:1033E0009F1CA5E0CA16D10481F6EB85FC8584916B
:1033F000FD858F9FF00D11242F0E311C2B853C85F0
:103400002F5F3F4F3C872B8735E0430E511C8DE2E9
:103410004816510409F077CF112319F01150109379
:10342000470280914D028F5F80934D02853080F07E
:1034300080914C0293E090934D0290910C01890F82
:1034400080934C028E5F853018F0919590930C011B
:1034500080E80E94000B882339F080914B02811193
:10346000CFC084E080934B0280E10E94000B882350
:1034700039F080914B02843009F0C4C010924B02A5
:1034800080914B02482F50E020914A02022E000CFE
:10349000330B4217530714F480934A0220914A02D7
:1034A000022E000C330B2E5F3F4F241735071CF400
:1034B000825080934A028AE0E1E2F1E0DE01119657
:1034C00001900D928A95E1F700914C02002E000CBC
:1034D000110B025E1F4FA12CB6E1EB2EF12C88E2FE
:1034E000C82ED12CB0904A02BA0C94E09B1540F142
:1034F00080914B02B81207C041E0B7016D5F7F4F6A
:10350000C8010E94B00CD0925502C0925402F092B1
:103510005702E0925602EB2DF0E0EE0FFF1FA1E004
:10352000B0E0AC0FBD1FEA0FFB1F808191810E94AC
:10353000D90EA394BAE0EB0EF11CE3E0AE12D2CFA9
:103540008BE598E00E94C012E6E3EE2EF12C0AE330
:1035500010E02CE330E04EE350E06CE370E086E3F3
:1035600090E00E949409FCE3EF2EF12C06E410E0B9
:1035700026E330E04AE450E066E370E082E490E065
:103580000E94940984E00E94000B882351F08091EE
:103590004B0281113BC010924902109248020E94D6
:1035A000DE110E94160B21CD10920F0110920E0118
:1035B00097FD0196959587959195819591099093A1
:1035C0004F0280934E0280910D01882331F068E212
:1035D00070E088E790E00E94070980914E02909188
:1035E0004F020196039708F053CE10924F021092AB
:1035F0004E0281E0809350024BCE70E060E0B7CE87
:10360000815030CF8F5F80934B023ACF813039F4B5
:1036100081E090E09093490280934802C0CF8230CD
:1036200039F481E090E090935D0280935C02B9CF21
:10363000833019F482E090E0F6CF843009F0B1CF06
:1036400083E090E0F0CF8BE290E09093550280937E
:10365000540281E090E090935702809356028DE1EE
:1036600098E00E946C0C04E110E010935502009366
:1036700054028BE090E090935702809356028DE0C5
:1036800098E00E946C0C8AE190E090935502809340
:10369000540285E190E0909357028093560281E0B6
:1036A00098E00E946C0C80914502909146020E9425
:1036B000150F10935502009354028FE190E0909300
:1036C00057028093560281EF97E00E946C0C88EEBF
:1036D00097E00E942C0E8FED97E00E94C01280911F
:1036E000440281116FC088E00E940B0B882309F40B
:1036F0004CC08091420290914302843B910528F492
:1037000001969093430280934202E0904202F0902F
:10371000430201E026E048E26AE270E08CE290E0D9
:103720000E94380D9701A8E2B0E00E94F62724EB32
:1037300030E040E050E00E94A227422F26E06AE2FB
:1037400070E08CE290E00E94160DF4EBEF16F104AD
:10375000E0F0109246021092450260E090E080E0B6
:103760000E94181080910D01882331F06CE271E005
:1037700080E590E00E94070981E08093440284EB99
:1037800090E0909343028093420284E00E94000BF9
:10379000882309F406CF109243021092420210923D
:1037A000440282EE9FEF90930F0180930E011092DE
:1037B0004F0210924E021092500210925D0210922F
:1037C0005C02EFCE01E026E048E26AE270E08CE2C3
:1037D00090E00E94380D26E048E26AE270E08CE258
:1037E00090E00E94160D8CE290E090935502809339
:1037F000540280E290E0909357028093560287ED46
:1038000097E00E946C0CC1CF80914D028F5F809336
:103810004D02853080F080914C0293E090934D02F0
:1038200090910C01890F80934C028E5F853018F0C7
:10383000919590930C0180E80E94000B882341F041
:1038400080914102882309F4D0C0815080934102C5
:1038500080E10E94000B882351F08091410290E0AA
:10386000019663E070E00E94342B80934102009146
:103870004C02002E000C110B025E1F4F88E290E0FC
:10388000909355028093540282E090E09093570207
:10389000809356028EEC97E00E946C0C84E190E0DD
:1038A00090935502809354022CE030E030935702FD
:1038B000209356028EEB97E00E946C0CF090410230
:1038C000F11006C041E069E170E0C8010E94B00C4F
:1038D00088E290E0909355028093540286E190E054
:1038E000909357028093560286EB97E00E946C0CEF
:1038F000D090100183EB97E0D11002C08FEA97E0DF
:103900000E946C0C31E0F31206C041E063E270E00B
:10391000C8010E94B00C88E290E090935502809319
:10392000540280E290E0909357028093560287EA17
:1039300097E00E946C0CE0900D0184EA97E0E110A2
:1039400002C080EA97E00E946C0C82E0F81206C088
:1039500041E06DE270E0C8010E94B00C88E290E0A6
:1039600090935502809354028AE290E0909357021C
:103970008093560286E997E00E946C0C10910B012F
:103980008FE797E0111102C08BE797E00E946C0C63
:103990008DE897E00E942C0E82E897E00E94C0120A
:1039A00088E00E94000B8823D1F0F11020C061E074
:1039B0006D256093100181E090E00E9418108091C5
:1039C000100181110AC00E945608809110018111D6
:1039D00004C080910D01882301F10E944D0984E00B
:1039E0000E94000B8111DDCEDCCD82E02FCF91E073
:1039F000F91209C06E2D6F2560930D0182E090E0F1
:103A00000E941810E2CFA2E0FA12DFCF61E0612736
:103A100060930B0183E090E0F3CF0E944809DFCF71
:103A200088E290E0909355028093540288E090E001
:103A3000909357028093560281E797E00E946C0CA6
:103A400080E390E0909355028093540282E190E0ED
:103A500090935702809356028AE697E00E946C0C7E
:103A60000091090110910A017AE1C72E77E0D72E63
:103A70005801B6E2AB1ABEEFBB0A7801F6016491B9
:103A8000C70105968538910570F4F0925502E092D1
:103A9000540224E230E0309357022093560283EE22
:103AA00096E00E94000C36E0E30EF11C8FEFC81A7E
:103AB000D80AAE14BF0411F780914002882321F088
:103AC0008150809340020AC00150110906329EEFD6
:103AD0001907BCF010930A010093090181E197E0F6
:103AE0000E942C0E84E00E94000B882309F459CD1B
:103AF00080E890E090930A018093090110924002BF
:103B000050CE80E890E090930A01809309018EE105
:103B1000D8CF80913E02882369F088E00E940B0B89
:103B200081113FCD84E00E940B0B81113ACD1092A0
:103B30003E0237CD80915A02882341F088E00E94EE
:103B40000B0B81112ECD10925A022BCD84E00E94D6
:103B5000000B882329F010925B0288E090E063CD8F
:103B600000913F0210E080913C0290913D02892B30
:103B700009F065C02FE832EC45EF5CE36091380254
:103B80007091390280913A0290913B020E9406287E
:103B9000609338027093390280933A0290933B020B
:103BA0000E94432A20E030E040E85FE30E940628BC
:103BB00020E030E040E05FE30E94D62920E030E0E2
:103BC00048E052E40E94D62920E030E048E851E481
:103BD0000E9406286B017C01A2E1A09FF001A19F39
:103BE000F00D1124E855FE4FC482D582E682F7829B
:103BF00088E00E94000B882311F1C0920501D09249
:103C00000601E0920701F092080181E090E09093B4
:103C10003D0280933C021092A7011092A60190935E
:103C200004018093030180910D01882309F4B9CC2C
:103C300068E270E088E592E00E940709B2CCB2E148
:103C4000B09FF001B19FF00D1124E855FE4FC080E8
:103C5000D180E280F38020E030E040EA50E4C70108
:103C6000B6010E94722887FDB5C020E030E046EF23
:103C700052E4C701B6010E94D129181634F4C12CB0
:103C8000D12C66EFE62E62E4F62E22E1209FF001B1
:103C9000219FF00D1124E855FE4FC082D182E282AF
:103CA000F3820E94E10D0E94BC0D0E9456100E94FA
:103CB0001F0F80913C0290913D02019709F087C04F
:103CC0008091030190910401880F991F2091A60112
:103CD0003091A701820F931F9093A7018093A601B3
:103CE0008436910564F084E690E09093A701809378
:103CF000A6018FEF9FEF90930401809303018091C1
:103D0000A6019091A7011816190654F01092A70168
:103D10001092A60181E090E090930401809303014A
:103D200080910B01882359F08091A6019091A70101
:103D30008D9666E070E0880F991F0E94070988E061
:103D40000E94000B882309F442C06091A601709183
:103D5000A7017093A5016093A401A2E1A09FC001F7
:103D6000A19F900D11248C0108551E4F072E000CA9
:103D7000880B990B0E94212920E030E048EC52E4A6
:103D80000E94772820E030E040E450E40E94D629E9
:103D90002AE939E949E95FE30E940628F8016087CA
:103DA0007187828793871486158616861786809179
:103DB0000D01882331F068E270E084E893E00E940E
:103DC000070986E090E090935D0280935C020E9478
:103DD0006D0DE7CBC12CD12C50EAE52E50E4F52E29
:103DE00054CF0E94E10D0E94BC0D0E9456100E940B
:103DF0001F0F0E946D0D84E00E94000B8F8B8111BC
:103E0000AACEB0913F02BB8B1B86EB850E2F10E034
:103E1000F2E1F09FC001F19F900D11249C01285503
:103E20003E4F5901D9015196BC91B98BBB2349F141
:103E3000F901C084D184E284F384C701B6019F777D
:103E40002DEC3CEC4CE45DE30E94722887FFACC291
:103E5000D5011C966D917D918D919C911F979F77B7
:103E60002DEC3CEC4CE45DE30E94722887FF9CC281
:103E7000F501148615861686178610861186128619
:103E800013862B852F5F2B873B89321708F0BDCF18
:103E900080E0D0903F02D81608F4B0C391E0980FAC
:103EA000998F9B87A2E1A89FC0011124FC01E855CE
:103EB000FE4F1F019F012F5E3F4F38A72FA3CF0159
:103EC00004969A8B898BDF011896BCA3ABA33C9612
:103ED000FEA3EDA380913F02FB858F1708F46EC30C
:103EE000AFA1B8A58C91882309F45AC2EF2FF0E056
:103EF000FE87ED8722E12E9F80012F9F100D112458
:103F000008551E4FD80151968C91882309F448C258
:103F1000D1018D919D910D90BC91A02D8B8F9C8F87
:103F2000AD8FBE8F9C01AD01F801608171818281EE
:103F300093810E9405282B013C01A989BA898D91A2
:103F40009D910D90BC91A02D8F8F98A3A9A3BAA38A
:103F50009C01AD01F80164817581868197810E9481
:103F600005284B015C01A3019201C301B2010E942B
:103F7000D6296B017C01A5019401C501B4010E9401
:103F8000D6299B01AC01C701B6010E9406280E94F8
:103F9000512A6B017C0120E030E040E850E40E94AF
:103FA000722887FFFDC120E030E0A901C701B601FA
:103FB0000E94D12918160CF0F3C1A7019601C30184
:103FC000B2010E9477282B013C01A7019601C5018F
:103FD000B4010E9477286B8B7C8B8D8B9E8BA70105
:103FE000960160E070E080E890E40E94052820E0FF
:103FF00030E040E05FE30E94D6294B015C01AC0158
:104000009B01C301B2010E94D6296B017C01AC0166
:104010009B016B8D7C8D8D8D9E8D0E940528D1011D
:104020006D937D938D939C931397A50194016B8958
:104030007C898D899E890E94D6294B015C01AC0147
:104040009B016F8D78A189A19AA10E940528E98919
:10405000FA896083718382839383A7019601D801D3
:104060006D917D918D919C910E940628F80160834D
:10407000718382839383A501940164817581868114
:1040800097810E940628D80114966D937D938D9395
:104090009C931797F101C080D180E280F38020E0EB
:1040A00030E040EA50E4C701B6010E94722887FD63
:1040B00087C220E030E046EF52E4C701B6010E941B
:1040C000D129181634F4C12CD12C26EFE22E22E48B
:1040D000F22ED101CD92DD92ED92FC921397E989F7
:1040E000FA89C080D180E280F38020E030E048E8A7
:1040F00051E4C701B6010E94722887FD68C220E022
:1041000030E04CE452E4C701B6010E94D1291816F0
:1041100034F4C12CD12C8CE4E82E82E4F82EA98949
:10412000BA89CD92DD92ED92FC92139782E12D85B2
:104130003E85829FF001839FF00D1124E855FE4FCC
:10414000C080D180E280F38020E030E040EA50E49B
:10415000C701B6010E94722887FD40C220E030E00E
:1041600046EF52E4C701B6010E94D129181634F473
:10417000C12CD12C16EFE12E12E4F12E22E1AD85F7
:10418000BE852A9FF0012B9FF00D1124E855FE4FAC
:10419000C082D182E282F382C480D580E680F7803B
:1041A00020E030E048E851E4C701B6010E947228DF
:1041B00087FD1BC220E030E04CE452E4C701B601A9
:1041C0000E94D129181634F4C12CD12CACE4EA2E6B
:1041D000A2E4FA2EA2E18D859E85A89F8001A99F69
:1041E000100D112408551E4FF801C482D582E682B5
:1041F000F782ABA1BCA18D909D90AD90BC90ADA17C
:10420000BEA18D919D910D90BC91A02D8D879E8713
:10421000AF87B88B2085318542855385C501B401B0
:104220000E940528A30192010E94D6296B017C01FE
:10423000F80124853585468557856D857E858F8572
:1042400098890E9405282B893C894D895E890E94A6
:10425000D6299B01AC01C701B6010E9406286B015B
:104260007C0120E030E0A9010E94D12918160CF051
:1042700097C0A7019601C301B2010E94D62920E090
:1042800030E040E05FE30E94D6292B013C01AC0105
:104290009B01C501B4010E940528ABA1BCA16D938F
:1042A0007D938D939C931397A70196016B897C89CD
:1042B0008D899E890E94D62920E030E040E05FE3AE
:1042C0000E94D6294B015C01AC019B016D857E8566
:1042D0008F8598890E940528EDA1FEA160837183D6
:1042E00082839383A3019201D80118966D917D91E9
:1042F0008D919C911B970E940628F8016087718719
:1043000082879387A5019401648575858685978545
:104310000E940628D8011C966D937D938D939C93E3
:104320001F9720E030E040E450E4C701B6010E944E
:10433000D6290E94F028662309F45EC1653008F092
:1043400064E083E0860F80936002C62ED12C460184
:10435000BFEF8B1A9B0A092C000CAA08BB08D1944A
:10436000C194D1080D2C000CEE08FF08A5019401A2
:10437000C701B6010E942C1060935F02A501940151
:10438000C701B6010E942C1060935E0280910D015E
:10439000882331F068E070E08CED90E00E9407091E
:1043A000EB85EF5FEB8796CDB2E1B09FC001B19F87
:1043B000900D1124FC01E855FE4F1F012081318131
:1043C00042815381C701B6010E9406282B013C019E
:1043D000D1014D925D926D927C9213971C968D90B7
:1043E0009D90AD90BC901F9714962D913D914D914D
:1043F0005C911797C501B4010E9406286D877E87DE
:104400008F87988BF101648375838683978320E07F
:1044100030E040EA50E4C301B2010E94722887FFF5
:1044200023C080E090E0A0EAB0E4F10180839183B2
:10443000A283B38320E030E0A901C701B6010E9446
:10444000722887FF2DC0C701B60190582DEC3CECB7
:104450004CEC5EE30E94D629D10118966D937D93B2
:104460008D939C931B971CC020E030E046EF52E4F4
:10447000C301B2010E94D129181694F480E090E0A3
:10448000A6EFB2E4F10180839183A283B38320E09D
:1044900030E0A901C701B6010E94D12918169CF28B
:1044A00020E030E048E851E46D857E858F8598896D
:1044B0000E94722887FF2CC0B2E1B09FC001B19F5B
:1044C000900D1124FC01E855FE4F7F0180E090E043
:1044D000A8E8B1E484839583A683B78320E030E025
:1044E000A901C501B4010E94722887FF38C0C50127
:1044F000B40190582DEC3CEC4CEC5EE30E94D629C4
:10450000D7011C966D937D938D939C931F9727C025
:1045100020E030E04CE452E46D857E858F859889FB
:104520000E94D1291816DCF4B2E1B09FC001B19FFE
:10453000900D1124FC01E855FE4F7F0180E090E0D2
:10454000ACE4B2E484839583A683B78320E030E0B3
:10455000A901C501B4010E94D129181644F2B2E1A3
:10456000B09FC001B19F900D1124FC01E855FE4F92
:104570007F0126EF38E24CE75FE360857185828535
:1045800093850E94D629D70118966D937D938D93BC
:104590009C931B9726EF38E24CE75FE31C966D91E6
:1045A0007D918D919C911F970E94D629F701648778
:1045B000758786879787F989FF8B63CC898D69CC4E
:1045C000C12CD12C90EAE92E90E4F92E82CDC12C99
:1045D000D12C08E8E02E01E4F02EA1CDC12CD12C85
:1045E000B0EAEB2EB0E4FB2EC9CDC12CD12CF8E8FB
:1045F000EF2EF1E4FF2EEECD61E0A3CEFF89F111A5
:104600000C94D11A8091A30190E0FC01EF55FE4F6C
:1046100020812F5F2083D394D0923F0260910201CA
:10462000E1EAF1E020E0621362C008EA11E0C12C87
:10463000CD1408F0B7C0D80151968C9151978823BA
:1046400009F451C020E030E048ED52E46D917D91D5
:104650008D919C910E9405282B013C0120E030E0C7
:1046600048E052E4F80164817581868197810E9457
:1046700005284B015C01A3019201C301B2010E9414
:10468000D6292B013C01A5019401C501B4010E946A
:10469000D6299B01AC01C301B2010E9406280E94E9
:1046A000512A4B015C0120E030E040E850E40E94D8
:1046B0007228181614F520E030E040E151E4C501FD
:1046C000B4010E94722818160CF05CC020E030E0A3
:1046D00040E651E4C501B4010E947228E9E1EE2EE2
:1046E000F12C18166CF4C3940E5E1F4FA1CF3191BC
:1046F000343008F40AC32F5F96CF74E6E72EF12C0E
:1047000020E030E040E850E4C501B4010E940528F3
:104710009F7720E030E040E05FE30E94722887FD51
:1047200035C020E030E040E151E4C501B4010E9411
:1047300005289F7720E030E040E05FE30E94722888
:1047400087FD28C020E030E040E651E4C501B40117
:104750000E9405289F7720E030E040E05FE30E9460
:10476000722887FD1BC0D8015096EC91F0E0EE0F47
:10477000FF1FE356FE4F80819181E80EF91EF18202
:10478000E082B1CF62E3E62EF12CBACF52E3E52E00
:10479000F12CE9CF49E1E42EF12CE5CF3CE0E32E0A
:1047A000F12CE1CF60919D0170919E0180914802B2
:1047B00090914902019741F480919F019091A0014D
:1047C000681779070CF4BC0180914502909146026C
:1047D000861797075CF481E080939C0170934602F2
:1047E0006093450290E080E00E94181087E090E01E
:1047F0000C94131BE0904802F0904902B1E0EB16D4
:10480000F10409F08DC220919D0130919E018091AB
:104810009F019091A0018217930744F102E010E0FC
:10482000281739072CF120E044E150E068E270E0FD
:104830008FE00E94930F21E044E150E064E370E0D8
:1048400085E00E94930F22E044E150E060E470E0D4
:1048500082E00E94930F23E044E150E06CE470E0BA
:1048600088E00E94930F10E000E066C001E010E0D5
:1048700020E048E050E064E170E080E00E94930FA7
:1048800021E048E050E060E270E081E00E94930F98
:1048900022E048E050E06CE270E082E00E94930F7A
:1048A00023E048E050E068E370E083E00E94930F6B
:1048B00024E048E050E064E470E084E00E94930F5C
:1048C00025E048E050E060E570E085E00E94930F4D
:1048D00086E00130110509F087E026E048E050E06D
:1048E00060E670E00E94930F27E04CE150E066E242
:1048F00070E088E00E94930F28E04CE150E062E312
:1049000070E089E00E94930F29E04CE150E06EE3F3
:1049100070E08AE00E94930F2AE04CE150E06AE4E4
:1049200070E08BE00E94930F2BE04CE150E066E5D5
:1049300070E08CE00E94930F88E097E00E942C0EBC
:1049400084E00E94000B882331F010929C011092A9
:104950005D0210925C0280919D0190919E01E11494
:10496000F10489F0EA94EF2811F00C94D11A0115A2
:10497000110511F40C94D11A000F111FF801E5561E
:10498000FE4F808191810E94EB0E0C94D11A809190
:104990003E02811112C084E00E94000B882369F05E
:1049A00081E080933E0280919B018093A3010E944D
:1049B000F60D85E090E00C94131B80919901909185
:1049C0009A01019690939A018093990142E088326E
:1049D000910528F044E08A35910508F048E02091DF
:1049E000980121113FC0242F30E0B9010E94202BF3
:1049F000892BE9F4809197018F5F877080939701ED
:104A000080910D01882399F0453088F448E3429F56
:104A1000C001439F900D921B112466E070E0805509
:104A20009B4F0E9407098091980181111BC08091C2
:104A3000990190919A0187399105A0F081E08093C6
:104A4000980180919B018823E9F086E0809397018B
:104A500080910D01882331F060E570E088E592E0F7
:104A60000E940709E0919701E730C0F4F0E0E55CAF
:104A7000FA4D0C94482B4425AC25B125B625B1251B
:104A8000AC25442580E0E2CF08E028E04DED56E07B
:104A90006EE070E08EE390E00E94400587E290E0D7
:104AA000909355028093540210925702109256022E
:104AB0008EEF96E00E946C0C81E590E09093550299
:104AC0008093540288E390E09093570280935602BB
:104AD00085EF96E00E946C0C80919801882311F478
:104AE0000C94D11A80919501909196010196909322
:104AF00096018093950185E190E090935502809313
:104B000054028EE190E090935702809356028DEE0E
:104B100096E00E946C0C80919B0190E001960E94AF
:104B2000150F85EE96E00E946C0C80919501909196
:104B300096018836914038F484E00E94000B882367
:104B400011F40C94D11A80919B018093A3011092CF
:104B50009601109295012BCF08E028E045ED56E034
:104B600097CF08E028E04DEC56E092CF21E046E0F8
:104B70006FE070E082E490E00E94870C8FCF0E948B
:104B8000E10D0E94BC0D0E9456100E941F0F01E013
:104B900020E440E870E060E090E080E00E94160DC4
:104BA00010920101C12C0EE010E08CE1E82EF12CF6
:104BB000D0905B02CD1008C040E0B8016E5F7F4F1F
:104BC00084E190E00E94B00CF0925502E092540211
:104BD00010935702009356028EEB96E0CC2039F0EA
:104BE00021E081EB96E0C21611F084EA96E00E9483
:104BF0006C0CC394045F1F4F33E0C312D9CF81E024
:104C00008093010180E80E94000B882339F08FEF28
:104C10008D0DD11001C082E080935B0280E10E9483
:104C2000000B882351F080915B0290E0019663E0D5
:104C300070E00E94342B80935B0288E00E94000B9E
:104C4000882389F080915B02811120C081E08093EC
:104C50005A020E943A0E8823B1F086E090E09093C9
:104C60005D0280935C0284E00E94000B882311F4B3
:104C70000C94D11A0E943A0E882309F49ACE86E049
:104C800090E00C94131B85E090E0E9CF813019F49B
:104C900089E090E0E4CF823031F78AE090E0DFCF26
:104CA0000E94E10D0E94BC0D0E9456100E941F0F31
:104CB00089E299E00E944D1288E00E94000B88234F
:104CC00029F081E080935A020E94DE1184E00E9464
:104CD000000B882311F40C94D11A0C94AD1D0E9482
:104CE000E10D0E94BC0D0E9456100E941F0F8BE127
:104CF00099E00E944D1288E00E94000B882331F356
:104D000010925D0210925C02E1CF019670E00E9469
:104D1000342B8093A3011092A5011092A40147CED9
:104D200010919C0120E048E050E06EE270E083E0EA
:104D30000E94930F21E048E050E06AE370E08DE0CC
:104D40000E94930F22E048E050E066E470E08EE0BD
:104D50000E94930F23E040E250E011111CC068E272
:104D600070E081E00E94930F24E040E250E064E3B1
:104D700070E08DE00E94930F25E040E250E060E497
:104D800070E08BE00E94930F26E040E250E06CE47C
:104D900070E084E066CD6EE270E088E00E94930FE0
:104DA00024E040E250E06AE370E089E00E94930F63
:104DB00025E040E250E066E470E08AE052CD8F9258
:104DC0009F92AF92BF92CF92DF92EF92FF92CF93DA
:104DD000DF93EC01688179818A819B81611571057E
:104DE0008105910521F464E279ED8BE597E02DE1F1
:104DF00033EF41E050E00E94A22749015A019B0194
:104E0000AC01A7EAB1E40E94C1276B017C01ACEEC2
:104E1000B4EFA50194010E94CF27C60ED71EE81E4D
:104E2000F91EF7FE06C081E0C81AD108E10880E843
:104E3000F80AC882D982EA82FB82C701B6019F774D
:104E4000DF91CF91FF90EF90DF90CF90BF90AF9028
:104E50009F908F9008958F929F92AF92BF92CF9222
:104E6000DF92EF92FF9260911D0170911E0180917F
:104E70001F0190912001611571058105910521F4B3
:104E800064E279ED8BE597E02DE133EF41E050E00E
:104E90000E94A22749015A019B01AC01A7EAB1E493
:104EA0000E94C1276B017C01ACEEB4EFA501940117
:104EB0000E94CF27C60ED71EE81EF91EF7FE06C0B9
:104EC00081E0C81AD108E10880E8F80AC0921D0103
:104ED000D0921E01E0921F01F0922001C701B6019D
:104EE0009F77FF90EF90DF90CF90BF90AF909F9013
:104EF0008F90089560931D0170931E0180931F0190
:104F0000909320010895FC0105900020E9F7809519
:104F100090958E0F9F1F0895F999FECF92BD81BD88
:104F2000F89A992780B50895262FF999FECF1FBAD0
:104F300092BD81BD20BD0FB6F894FA9AF99A0FBEC2
:104F400001960895052E97FB1EF400940E94B92740
:104F500057FD07D00E94D42707FC03D04EF40C94D1
:104F6000B92750954095309521953F4F4F4F5F4F52
:104F7000089590958095709561957F4F8F4F9F4FC5
:104F800008950E94F627A59F900DB49F900DA49FB1
:104F9000800D911D11240895B7FF0C94C1270E9424
:104FA000C127821B930B0895A1E21A2EAA1BBB1BDB
:104FB000FD010DC0AA1FBB1FEE1FFF1FA217B307E5
:104FC000E407F50720F0A21BB30BE40BF50B661FFB
:104FD000771F881F991F1A9469F7609570958095BF
:104FE00090959B01AC01BD01CF010895A29FB00136
:104FF000B39FC001A39F700D811D1124911DB29F0D
:10500000700D811D1124911D08955058BB27AA27AA
:105010000E941D280C9497290E94892938F00E942B
:10502000902920F039F49F3F19F426F40C94862936
:105030000EF4E095E7FB0C948029E92F0E94A82943
:1050400058F3BA17620773078407950720F079F4BD
:10505000A6F50C94CA290EF4E0950B2EBA2FA02DBC
:105060000B01B90190010C01CA01A0011124FF2715
:10507000591B99F0593F50F4503E68F11A16F04010
:10508000A22F232F342F4427585FF3CF469537950F
:105090002795A795F0405395C9F77EF41F16BA0BD4
:1050A000620B730B840BBAF09150A1F0FF0FBB1F82
:1050B000661F771F881FC2F70EC0BA0F621F731FCB
:1050C000841F48F4879577956795B795F7959E3F28
:1050D00008F0B0CF9395880F08F09927EE0F9795B9
:1050E000879508950E945C2908F481E008950E9444
:1050F0008B280C9497290E94902958F00E948929A6
:1051000040F029F45F3F29F00C94802951110C9450
:10511000CB290C9486290E94A82968F39923B1F31E
:10512000552391F3951B550BBB27AA2762177307CD
:10513000840738F09F5F5F4F220F331F441FAA1F61
:10514000A9F335D00E2E3AF0E0E832D0915050401D
:10515000E695001CCAF72BD0FE2F29D0660F771FCB
:10516000881FBB1F261737074807AB07B0E809F0B1
:10517000BB0B802DBF01FF2793585F4F3AF09E3F36
:10518000510578F00C9480290C94CB295F3FE4F30F
:10519000983ED4F3869577956795B795F7959F5F79
:1051A000C9F7880F911D9695879597F90895E1E0C5
:1051B000660F771F881FBB1F621773078407BA0724
:1051C00020F0621B730B840BBA0BEE1F88F7E0957F
:1051D00008950E94F0286894B1110C94CB29089589
:1051E0000E94B02988F09F5798F0B92F9927B7519E
:1051F000B0F0E1F0660F771F881F991F1AF0BA957B
:10520000C9F714C0B13091F00E94CA29B1E00895E5
:105210000C94CA29672F782F8827B85F39F0B93FD7
:10522000CCF3869577956795B395D9F73EF490952D
:105230008095709561957F4F8F4F9F4F0895E894AB
:1052400009C097FB3EF490958095709561957F4FCE
:105250008F4F9F4F9923A9F0F92F96E9BB2793957C
:10526000F695879577956795B795F111F8CFFAF48C
:10527000BB0F11F460FF1BC06F5F7F4F8F4F9F4FBD
:1052800016C0882311F096E911C0772321F09EE81B
:10529000872F762F05C0662371F096E8862F70E081
:1052A00060E02AF09A95660F771F881FDAF7880F5B
:1052B0009695879597F90895990F0008550FAA0BB1
:1052C000E0E8FEEF16161706E807F907C0F0121619
:1052D0001306E407F50798F0621B730B840B950B1C
:1052E00039F40A2661F0232B242B252B21F4089571
:1052F0000A2609F4A140A6958FEF811D811D08950E
:1053000097F99F6780E870E060E008959FEF80EC78
:10531000089500240A94161617061806090608951B
:1053200000240A9412161306140605060895092E81
:105330000394000C11F4882352F0BB0F40F4BF2BF0
:1053400011F460FF04C06F5F7F4F8F4F9F4F089530
:1053500057FD9058440F551F59F05F3F71F0479526
:10536000880F97FB991F61F09F3F79F0879508950B
:10537000121613061406551FF2CF4695F1DF08C02A
:10538000161617061806991FF1CF86957105610547
:1053900008940895E894BB2766277727CB0197F9EF
:1053A00008950E945C2908F48FEF08950E94E9296E
:1053B0000C9497290E94892938F00E94902920F0A6
:1053C000952311F00C9480290C94862911240C94B7
:1053D000CB290E94A82970F3959FC1F3950F50E047
:1053E000551F629FF001729FBB27F00DB11D639F97
:1053F000AA27F00DB11DAA1F649F6627B00DA11D3D
:10540000661F829F2227B00DA11D621F739FB00DE2
:10541000A11D621F839FA00D611D221F749F332752
:10542000A00D611D231F849F600D211D822F762FEB
:105430006A2F11249F5750409AF0F1F088234AF0C8
:10544000EE0FFF1FBB1F661F771F881F9150504034
:10545000A9F79E3F510580F00C9480290C94CB292C
:105460005F3FE4F3983ED4F3869577956795B795BB
:10547000F795E7959F5FC1F7FE2B880F911D9695D5
:10548000879597F908959F930E94A82A0F9007FC8B
:10549000EE5F0C94D12A19F416F40C9486290C941E
:1054A000912A0E94B029B8F39923C9F3B6F39F5704
:1054B000550B87FF0E949F2A0024A0E640EA900136
:1054C00080585695979528F4805C660F771F881F43
:1054D00020F026173707480730F4621B730B840B44
:1054E000202931294A2BA695179407942025312588
:1054F0004A2758F7660F771F881F20F026173707AF
:10550000480730F4620B730B840B200D311D411DD5
:10551000A09581F7B901842F9158880F96958795AA
:1055200008959F3F31F0915020F4879577956795C6
:10553000B795880F911D9695879597F90895915085
:105540005040660F771F881FD2F708950C94862964
:105550000E94B029D8F3E894E0E0BB279F57F0F011
:105560002AED3FE049EC06C0EE0FBB0F661F771F28
:10557000881F28F0B23A62077307840728F0B25AEE
:10558000620B730B840BE3959A9572F7803830F4B5
:105590009A95BB0F661F771F881FD2F790480C940F
:1055A000932AEF93E0FF07C0A2EA2AED3FE049EC1F
:1055B0005FEB0E941D280E9497290F90039401FC25
:1055C0009058ECEAF0E00C94E52A9F938F937F9338
:1055D0006F93FF93EF939B01AC010E94D629EF914B
:1055E000FF910E94F92A2F913F914F915F910C9466
:1055F000D629DF93CF931F930F93FF92EF92DF9201
:105600007B018C01689406C0DA2EEF010E94E92923
:10561000FE01E894A5912591359145915591A6F308
:10562000EF010E941D28FE019701A801DA9469F795
:10563000DF90EF90FF900F911F91CF91DF91089530
:10564000AA1BBB1B51E107C0AA1FBB1FA617B707A8
:1056500010F0A61BB70B881F991F5A95A9F78095C4
:105660009095BC01CD01089597FB072E16F4009488
:1056700007D077FD09D00E94202B07FC05D03EF40F
:10568000909581959F4F0895709561957F4F0895EE
:10569000EE0FFF1F0590F491E02D09940E94F6276C
:0E56A000B7FF0895821B930B0895F894FFCF77
:1056AE001001010100000008428000010101E2FF2B
:1056BE0001FFFFFFFF00E1000000000000010000FD
:1056CE0000570160016A0174017D0100C1808100F3
:1056DE000000000000000207810623071807690773
:1056EE002707450700000000000C1508670E660E20
:1056FE00284229204E4F003120504C41594552002E
:10570E003220504C41594552530048494748534363
:10571E004F52450053455454494E475300494E4647
:02572E004F002A
:00000001FF
